Archive member included because of file (symbol)

F:/PROGRAMY/WinAVR/bin/../lib/gcc/avr/3.4.3\libgcc.a(_udivmodqi4.o)
                              clock.o (__udivmodqi4)
F:/PROGRAMY/WinAVR/bin/../lib/gcc/avr/3.4.3\libgcc.a(_copy_data.o)
                              clock.o (__do_copy_data)
F:/PROGRAMY/WinAVR/bin/../lib/gcc/avr/3.4.3\libgcc.a(_clear_bss.o)
                              clock.o (__do_clear_bss)

Memory Configuration

Name             Origin             Length             Attributes
text             0x00000000         0x00002000         xr
data             0x00800060         0x0000ffa0         rw !x
eeprom           0x00810000         0x00010000         rw !x
*default*        0x00000000         0xffffffff

Linker script and memory map

LOAD F:/PROGRAMY/WinAVR/bin/../lib/gcc/avr/3.4.3/../../../../avr/lib/crttn26.o
LOAD clock.o
LOAD F:/PROGRAMY/WinAVR/bin/../lib/gcc/avr/3.4.3/../../../../avr/lib\libm.a
LOAD F:/PROGRAMY/WinAVR/bin/../lib/gcc/avr/3.4.3\libgcc.a
LOAD F:/PROGRAMY/WinAVR/bin/../lib/gcc/avr/3.4.3/../../../../avr/lib\libc.a
LOAD F:/PROGRAMY/WinAVR/bin/../lib/gcc/avr/3.4.3\libgcc.a

.hash
 *(.hash)

.dynsym
 *(.dynsym)

.dynstr
 *(.dynstr)

.gnu.version
 *(.gnu.version)

.gnu.version_d
 *(.gnu.version_d)

.gnu.version_r
 *(.gnu.version_r)

.rel.init
 *(.rel.init)

.rela.init
 *(.rela.init)

.rel.text
 *(.rel.text)
 *(.rel.text.*)
 *(.rel.gnu.linkonce.t*)

.rela.text
 *(.rela.text)
 *(.rela.text.*)
 *(.rela.gnu.linkonce.t*)

.rel.fini
 *(.rel.fini)

.rela.fini
 *(.rela.fini)

.rel.rodata
 *(.rel.rodata)
 *(.rel.rodata.*)
 *(.rel.gnu.linkonce.r*)

.rela.rodata
 *(.rela.rodata)
 *(.rela.rodata.*)
 *(.rela.gnu.linkonce.r*)

.rel.data
 *(.rel.data)
 *(.rel.data.*)
 *(.rel.gnu.linkonce.d*)

.rela.data
 *(.rela.data)
 *(.rela.data.*)
 *(.rela.gnu.linkonce.d*)

.rel.ctors
 *(.rel.ctors)

.rela.ctors
 *(.rela.ctors)

.rel.dtors
 *(.rel.dtors)

.rela.dtors
 *(.rela.dtors)

.rel.got
 *(.rel.got)

.rela.got
 *(.rela.got)

.rel.bss
 *(.rel.bss)

.rela.bss
 *(.rela.bss)

.rel.plt
 *(.rel.plt)

.rela.plt
 *(.rela.plt)

.text           0x00000000      0x304
 *(.vectors)
 .vectors       0x00000000       0x18 F:/PROGRAMY/WinAVR/bin/../lib/gcc/avr/3.4.3/../../../../avr/lib/crttn26.o
                0x00000000                __vectors
                0x00000000                __vector_default
                0x00000018                __ctors_start = .
 *(.ctors)
                0x00000018                __ctors_end = .
                0x00000018                __dtors_start = .
 *(.dtors)
                0x00000018                __dtors_end = .
 *(.progmem.gcc*)
 *(.progmem*)
                0x00000018                . = ALIGN (0x2)
 *(.init0)
 *(.init1)
 *(.init2)
 .init2         0x00000018        0x8 F:/PROGRAMY/WinAVR/bin/../lib/gcc/avr/3.4.3/../../../../avr/lib/crttn26.o
 *(.init3)
 *(.init4)
 .init4         0x00000020       0x18 F:/PROGRAMY/WinAVR/bin/../lib/gcc/avr/3.4.3\libgcc.a(_copy_data.o)
                0x00000020                __do_copy_data
 .init4         0x00000038       0x10 F:/PROGRAMY/WinAVR/bin/../lib/gcc/avr/3.4.3\libgcc.a(_clear_bss.o)
                0x00000038                __do_clear_bss
 *(.init5)
 *(.init6)
 *(.init7)
 *(.init8)
 *(.init9)
 .init9         0x00000048        0x2 F:/PROGRAMY/WinAVR/bin/../lib/gcc/avr/3.4.3/../../../../avr/lib/crttn26.o
 *(.text)
 .text          0x0000004a        0x2 F:/PROGRAMY/WinAVR/bin/../lib/gcc/avr/3.4.3/../../../../avr/lib/crttn26.o
                0x0000004a                __vector_1
                0x0000004a                __bad_interrupt
                0x0000004a                __vector_6
                0x0000004a                __vector_3
                0x0000004a                __vector_11
                0x0000004a                __vector_7
                0x0000004a                __vector_4
                0x0000004a                __vector_9
                0x0000004a                __vector_2
                0x0000004a                __vector_8
                0x0000004a                __vector_10
 .text          0x0000004c      0x2a0 clock.o
                0x000000de                minSet
                0x00000058                wait
                0x0000022c                __vector_5
                0x0000015e                main
                0x0000004c                delay
                0x0000006e                hourSet
                0x000002ec                . = ALIGN (0x2)
 *(.text.*)
 .text.libgcc   0x000002ec       0x18 F:/PROGRAMY/WinAVR/bin/../lib/gcc/avr/3.4.3\libgcc.a(_udivmodqi4.o)
                0x000002ec                __udivmodqi4
                0x00000304                . = ALIGN (0x2)
 *(.fini9)
 *(.fini8)
 *(.fini7)
 *(.fini6)
 *(.fini5)
 *(.fini4)
 *(.fini3)
 *(.fini2)
 *(.fini1)
 *(.fini0)
                0x00000304                _etext = .

.data           0x00800060        0xa load address 0x00000304
                0x00800060                PROVIDE (__data_start, .)
 *(.data)
 .data          0x00800060        0xa clock.o
                0x00800060                digit
 *(.gnu.linkonce.d*)
                0x0080006a                . = ALIGN (0x2)
                0x0080006a                _edata = .
                0x0080006a                PROVIDE (__data_end, .)

.bss            0x0080006a        0xd
                0x0080006a                PROVIDE (__bss_start, .)
 *(.bss)
 .bss           0x0080006a        0xd clock.o
                0x0080006d                msec
                0x0080006f                minSetCt
                0x00800075                waitCt
                0x00800074                hourSetF
                0x0080006a                hour
                0x0080006b                min
                0x0080006c                sec
                0x00800071                minSetF
                0x00800072                hourSetCt
 *(COMMON)
                0x00800077                PROVIDE (__bss_end, .)
                0x00000304                __data_load_start = LOADADDR (.data)
                0x0000030e                __data_load_end = (__data_load_start + SIZEOF (.data))

.noinit         0x00800077        0x0
                0x00800077                PROVIDE (__noinit_start, .)
 *(.noinit*)
                0x00800077                PROVIDE (__noinit_end, .)
                0x00800077                _end = .
                0x00800077                PROVIDE (__heap_start, .)

.eeprom         0x00810000        0x0
 *(.eeprom*)
                0x00810000                __eeprom_end = .

.stab
 *(.stab)

.stabstr
 *(.stabstr)

.stab.excl
 *(.stab.excl)

.stab.exclstr
 *(.stab.exclstr)

.stab.index
 *(.stab.index)

.stab.indexstr
 *(.stab.indexstr)

.comment
 *(.comment)

.debug
 *(.debug)

.line
 *(.line)

.debug_srcinfo
 *(.debug_srcinfo)

.debug_sfnames
 *(.debug_sfnames)

.debug_aranges  0x00000000       0x14
 *(.debug_aranges)
 .debug_aranges
                0x00000000       0x14 clock.o

.debug_pubnames
                0x00000000       0xbf
 *(.debug_pubnames)
 .debug_pubnames
                0x00000000       0xbf clock.o

.debug_info     0x00000000      0x1eb
 *(.debug_info)
 .debug_info    0x00000000      0x1eb clock.o
 *(.gnu.linkonce.wi.*)

.debug_abbrev   0x00000000       0xcb
 *(.debug_abbrev)
 .debug_abbrev  0x00000000       0xcb clock.o

.debug_line     0x00000000      0x2a3
 *(.debug_line)
 .debug_line    0x00000000      0x2a3 clock.o

.debug_frame
 *(.debug_frame)

.debug_str      0x00000000       0xef
 *(.debug_str)
 .debug_str     0x00000000       0xef clock.o
                                0x123 (size before relaxing)

.debug_loc
 *(.debug_loc)

.debug_macinfo
 *(.debug_macinfo)
OUTPUT(clock.elf elf32-avr)

Cross Reference Table

Symbol                                            File
__bad_interrupt                                   F:/PROGRAMY/WinAVR/bin/../lib/gcc/avr/3.4.3/../../../../avr/lib/crttn26.o
__bss_end                                         F:/PROGRAMY/WinAVR/bin/../lib/gcc/avr/3.4.3\libgcc.a(_clear_bss.o)
__bss_start                                       F:/PROGRAMY/WinAVR/bin/../lib/gcc/avr/3.4.3\libgcc.a(_clear_bss.o)
__data_end                                        F:/PROGRAMY/WinAVR/bin/../lib/gcc/avr/3.4.3\libgcc.a(_copy_data.o)
__data_load_start                                 F:/PROGRAMY/WinAVR/bin/../lib/gcc/avr/3.4.3\libgcc.a(_copy_data.o)
__data_start                                      F:/PROGRAMY/WinAVR/bin/../lib/gcc/avr/3.4.3\libgcc.a(_copy_data.o)
__do_clear_bss                                    F:/PROGRAMY/WinAVR/bin/../lib/gcc/avr/3.4.3\libgcc.a(_clear_bss.o)
                                                  clock.o
__do_copy_data                                    F:/PROGRAMY/WinAVR/bin/../lib/gcc/avr/3.4.3\libgcc.a(_copy_data.o)
                                                  clock.o
__heap_end                                        F:/PROGRAMY/WinAVR/bin/../lib/gcc/avr/3.4.3/../../../../avr/lib/crttn26.o
__init                                            F:/PROGRAMY/WinAVR/bin/../lib/gcc/avr/3.4.3/../../../../avr/lib/crttn26.o
__stack                                           F:/PROGRAMY/WinAVR/bin/../lib/gcc/avr/3.4.3/../../../../avr/lib/crttn26.o
                                                  clock.o
__udivmodqi4                                      F:/PROGRAMY/WinAVR/bin/../lib/gcc/avr/3.4.3\libgcc.a(_udivmodqi4.o)
                                                  clock.o
__vector_1                                        F:/PROGRAMY/WinAVR/bin/../lib/gcc/avr/3.4.3/../../../../avr/lib/crttn26.o
__vector_10                                       F:/PROGRAMY/WinAVR/bin/../lib/gcc/avr/3.4.3/../../../../avr/lib/crttn26.o
__vector_11                                       F:/PROGRAMY/WinAVR/bin/../lib/gcc/avr/3.4.3/../../../../avr/lib/crttn26.o
__vector_2                                        F:/PROGRAMY/WinAVR/bin/../lib/gcc/avr/3.4.3/../../../../avr/lib/crttn26.o
__vector_3                                        F:/PROGRAMY/WinAVR/bin/../lib/gcc/avr/3.4.3/../../../../avr/lib/crttn26.o
__vector_4                                        F:/PROGRAMY/WinAVR/bin/../lib/gcc/avr/3.4.3/../../../../avr/lib/crttn26.o
__vector_5                                        clock.o
                                                  F:/PROGRAMY/WinAVR/bin/../lib/gcc/avr/3.4.3/../../../../avr/lib/crttn26.o
__vector_6                                        F:/PROGRAMY/WinAVR/bin/../lib/gcc/avr/3.4.3/../../../../avr/lib/crttn26.o
__vector_7                                        F:/PROGRAMY/WinAVR/bin/../lib/gcc/avr/3.4.3/../../../../avr/lib/crttn26.o
__vector_8                                        F:/PROGRAMY/WinAVR/bin/../lib/gcc/avr/3.4.3/../../../../avr/lib/crttn26.o
__vector_9                                        F:/PROGRAMY/WinAVR/bin/../lib/gcc/avr/3.4.3/../../../../avr/lib/crttn26.o
__vector_default                                  F:/PROGRAMY/WinAVR/bin/../lib/gcc/avr/3.4.3/../../../../avr/lib/crttn26.o
__vectors                                         F:/PROGRAMY/WinAVR/bin/../lib/gcc/avr/3.4.3/../../../../avr/lib/crttn26.o
delay                                             clock.o
digit                                             clock.o
hour                                              clock.o
hourSet                                           clock.o
hourSetCt                                         clock.o
hourSetF                                          clock.o
main                                              clock.o
                                                  F:/PROGRAMY/WinAVR/bin/../lib/gcc/avr/3.4.3/../../../../avr/lib/crttn26.o
min                                               clock.o
minSet                                            clock.o
minSetCt                                          clock.o
minSetF                                           clock.o
msec                                              clock.o
sec                                               clock.o
wait                                              clock.o
waitCt                                            clock.o
